:1000000042C067C15AC059C058C057C056C055C039
:1000100054C053C052C051C050C04FC04EC04DC05C
:100020004CC04BC04AC004030904180372006100AD
:10003000700068006E00650074002E006E006500A0
:1000400074001203550053004200540065006E0016
:100050006B00690012010101FF0000088117980A76
:1000600001010102030109021200010100803209AD
:1000700004000000000000000E03420031003000C8
:1000800030003000320011241FBECFE5D4E0DEBFC7
:10009000CDBF10E0A0E6B0E0E6E5FAE002C00590D2
:1000A0000D92A436B107D9F710E0A4E6B0E001C084
:1000B0001D92A939B107E1F73BC3A2CF84E690E0D6
:1000C000809390000B9680938F0085B7836085BFE7
:1000D0008BB780648BBF08950F931F93CF93DF93EB
:1000E00080919500882309F493C0982F935097FD31
:1000F0008DC080918F00282F2F5FE90180919200A1
:100100008D3209F07DC0983009F07AC08881807600
:1001100009F068C02DE830E010928D0089818823B5
:1001200041F410928E00309394002093930092E05B
:1001300006C0853031F48A818093960090E020E8F3
:1001400057C08630B9F58B81813019F484E590E091
:1001500021C0823019F486E690E01CC0833009F09B
:1001600045C08A81882341F486E290E09093940010
:100170008093930094E03BC0813041F48AE290E0A8
:10018000909394008093930098E131C0823041F4C1
:1001900082E490E0909394008093930092E127C0D2
:1001A000833021F588E790E090939400809393004A
:1001B0009EE01DC0883039F488E990E09093940067
:1001C000809393000DC0893021F48A818093980038
:1001D000B5CF8A3009F0B2CF3093940020939300CA
:1001E00091E0ADCFCE01CBD2982FA9CF90E020ECFB
:1001F0008F81882339F48E81891720F4982F02C0CB
:1002000090E020E820937A0090936000109295008F
:10021000909160009F3F09F440C08091610084FF8D
:100220003CC0692F993008F068E0961B90936000FD
:1002300080917A0080FF02C003EC01C00BE48F5F65
:1002400080937A00E0919300F091940086FD04C0C1
:10025000962FA5E8B0E00CC0962FA5E8B0E003C04B
:1002600084918D9331969150D8F704C081918D93EC
:100270009150E0F7F0939400E09393007727162FC6
:1002800085E890E0C9D1183018F48FEF80936000B2
:10029000009384001C5F1093610080B3857019F097
:1002A00010927B0011C080917B00882369F494E652
:1002B00080B3857049F49150D9F781E080937B0039
:1002C0001092960010929100DF91CF911F910F91A3
:1002D00008950F930FB70F93809BFECF809B06C0AE
:1002E000809B04C0809B02C0000000C01F933F930E
:1002F0002F9331E014E000B3102710FD32E0102FEF
:100300003A95C9F700FDE3C000B3102720E010FBC9
:1003100020F9DF9310B3012700FB21F9CF93C0919F
:10032000900000B3102710FB22F93BE0D0E04F9380
:1003300010B3012700FB23F94FEF000055C0809B4D
:10034000FECF809B06C0809B04C0809B02C0000043
:1003500000C0DF9100C0CDCF10B3157079F14F7D93
:10036000206213C000B3057049F14F7B206415C0B3
:10037000057021F1102F206800B319C000B305707B
:10038000E9F04E7F216018C039F300B30570B1F079
:10039000102710FB26F9223028F310B3012700FBA9
:1003A00027F9422749934FEF00B3243008F3102771
:1003B00010FB20F9297F11F310B31570E1F101272B
:1003C00000FB21F9237FF1F000B30570A1F11027A4
:1003D00010FB22F9277EE1F010B3012700FB23F97F
:1003E0003A9541F12F7CD1F000B3057021F110272F
:1003F00010FB24F92F79C1F010B3012700FB25F978
:100400002F73C2CF10B31570B1F04D7F2260DCCFD7
:1004100000B3057081F04B7F2460DECF10B3157000
:1004200051F0477F2860E0CF00B3057021F04F7E88
:100430002061E2CF3BC03C2FC09190003C1B00E408
:1004400033300ABF98F108811981412F1F7720911D
:1004500091000D3279F1013E69F10936C1F007775B
:10046000033421F510919700112301F100919500BB
:100470000030C1F53430C2F13093950010939200F2
:1004800000918F00C0938F00009390002DC0121731
:1004900069F43091610034FD23C00AE500936100E6
:1004A000C4E8D0E025C00027009397004F91CF917A
:1004B000DF910DC01217B9F7009397000AE500937A
:1004C00061004F91CF910AB706FD39CFDF9100E46B
:1004D0000ABF2F913F911F910F910FBF0F91189558
:1004E000432F03C04AE501C042EDC4E1D0E032E051
:1004F0005F9355E0909A02B3889A8A9A20E80FC0D9
:10050000052710E002BB10C0052710E0089402BBCD
:1005100013C0052710E015C0052710E019C020FF03
:10052000052702BB279517951C3F50F720FF05278D
:10053000279502BB17951C3F38F720FF0527279505
:10054000179502BB1C3F28F720FF05272795179515
:100550001C3F02BB08F700C0499120FF052702BBE2
:10056000279517951C3F80F520FF0527279502BB8F
:1005700017951C3F68F520FF05272795179502BBA7
:100580001C3F58F520FF0527279517951C3F02BBF8
:1005900038F5242F3A9519F60A7F5F9102BB32E0B5
:1005A0003A95F1F710919600C651D04011F0109392
:1005B0009100016011B31A7F02BB0A7F4F91CF9166
:1005C00011BB02BBDF9183CF052710E002BBCACF6E
:1005D000052710E0089402BBCDCF052710E0CFCF50
:1005E000052710E0D3CFA82FB92F8FEF9FEF41E061
:1005F00050EA615070F02D9138E0722F782796956F
:100600008795269570FF02C0842795273A95A9F70C
:10061000F0CF809590950895E6DF8D939D93089592
:1006200085B3806385BB8FEF80B981B18C7F81B941
:1006300008950F931F93982FFA01D8016115710542
:1006400031F42115310571F52FEF3FEF5FC084EADA
:1006500086BF06B607FEFDCF81B1887F883019F0CE
:1006600021E030E053C0892F880F83B984E886BF2A
:1006700006B607FEFDCF81B1887F883109F042C000
:1006800044E807C0808183B946BF06B607FEFDCFA8
:100690003196615070408FEF6F3F780799F72115C1
:1006A000310559F184EA86BF06B607FEFDCF81B158
:1006B000803119F023E030E027C0990F916093B9A1
:1006C00084E886BF06B607FEFDCF81B1803479F09D
:1006D00024E030E019C02115310511F084EC01C08F
:1006E00084E886BF06B607FEFDCF83B18D93215007
:1006F00030408FEF2F3F380771F784E986BF20E045
:1007000030E004C022E030E084E986BFC9011F91D7
:100710000F910895FC0190E002C0819198276150EB
:1007200070408FEF6F3F7807C1F7892F99270895A1
:10073000CFE5D4E0DEBFCDBF88E190E02EE00FB67C
:10074000F894A89581BD0FBE21BD8FEF85BB14BA6B
:1007500067DF7DD1892B09F0FFCF88EF82BB85E071
:1007600081BB9EEF8FEF9150F1F78150E1F781B39C
:100770008A7F81BBA3DC7894A895AEDCFDCFCF92B5
:10078000DF92FF920F931F93CF93DF93EC011092B0
:1007900062008CE7C82E80E0D82ED0929400C092E0
:1007A0009300F98082E0F816D9F1E0E1FE1629F015
:1007B000F1E0FF1609F042C022C00A81112727D1BB
:1007C00008171907DCF5F0927C00B6016F5F7F4FC8
:1007D0008A812DD1EC0197FF05C010927C0081E049
:1007E00090E02EC08C010F5F1F4FB801C60192DF51
:1007F00004581F4FF8018083CE01029621C00A8160
:10080000112705D108171907CCF4F0927C008A81D2
:1008100001D180937D0062E070E08CE790E008C039
:10082000F0927C00F4D080937D0062E070E0C6011D
:1008300071DF80937E0083E090E002C080E090E072
:100840009927DF91CF911F910F91FF90DF90CF906B
:1008500008950000000000000000000000000000FB
:100860000000000000000000000000000000000088
:100870000000000000000000000000000000000078
:100880000000000000000000000000000000000068
:100890000000000000000000000000000000000058
:1008A0000000000000000000000000000000000048
:1008B0000000000000000000000000000000000038
:1008C0000000000000000000000000000000000028
:1008D0000000000000000000000000000000000018
:1008E0000000000000000000000000000000000008
:1008F00000000000000000000000000000000000F8
:1009000000000000000000000000000000000000E7
:1009100000000895A59AAD98A498AC9A08950F93F5
:100920001F93182FAD9A95DFAC98A49A92DFAD98DB
:1009300090DFAD9A8EDFA498AC9A8BDFAD9889DFFB
:1009400000E017FF03C0A498AC9A02C0AC98A49A28
:1009500080DFAD9A7EDFAD980F5F083011F0110F88
:10096000F0CFA498AC9A75DFAD9A73DF83B3AD98DE
:1009700084FF03C08FEF9FEF04C09C9BFECF80E0FD
:1009800090E01F910F910895EF92FF920F931F93A4
:10099000CF93DF937C01062F10E0C0E0D0E059DF59
:1009A000AD9A57DF110F9C991160AD982196C83010
:1009B000D105A9F7F7011083002311F4AC98A49A8C
:1009C00048DFAD9A46DFAD98A498AC9A42DF80E04C
:1009D00090E0DF91CF911F910F91FF90EF900895DC
:1009E000CF93DF93EB019BDF892B19F08FEF9FEF04
:1009F0000BC09C99FECF60E0CE01C6DF61E0CE0166
:100A00000196C2DF80E090E0DF91CF91089582E00F
:100A100090E00895882341F0813019F484E090E05B
:100A200008958FEF9FEF089583E090E00895882365
:100A300029F0813029F08FEF9FEF089583E001C006
:100A400085E0CEDF009711F482E090E0089562DF48
:060A500080E090E0089533
:040A5600FF5A010042
:00000001FF
